:0A0000005F2C0000000000005F2EDE
:04000A0000000800EA
:0C000E001030FD00FD0B09280000080068
:10001A000830FC002330FD00FD0B1128FC0B1128D1
:02002A000800CC
:10002C0083160313A61B1D28831286131F28831205
:10003C0086178316261B252883120613272883125E
:10004C0006178316A61A2D28831286122F288312C0
:10005C0086168316261A3528831206123728831221
:10006C000616DD183B2805173C28051385170520B7
:10007C0085138316A61945288312861347288312E5
:10008C008617831626194D28831206134F288312C0
:10009C0006178316A6185528831286125728831222
:1000AC008616831626185D28831206125F28831283
:1000BC000616DD1863280517642805138517052017
:0E00CC008513DD1C6B280D206C280720080012
:1000DA0083120313DD1083162508A6001620DD14EB
:0200EA0008000C
:1000EC0083120313FB01FA01F9018030F800F10CC3
:1000FC00F00C031C8A287408F90775080318750F8F
:10010C00FA070318FB0A0310F01F92287408FA0769
:10011C0075080318750FFB07FB0CFA0CF90CF80C9F
:10012C00031C7D287B08F3007A08F2007908F100A3
:06013C007808F000080045
:1001420083120313F8010830FC00700DF80D7408D7
:10015200F8020318AE28F8070310F00DFC0BA628CE
:02016200080093
:1001640083160313A201220883126F078400000878
:100174000319C8288316220883126F078400000815
:0E0184008316A5006D208316A20AB528080078
:10019200831603131208013EF000F1010318F10A5D
:1001A20083126F08F400F50176200630F200700821
:1001B200F4007108F50072080319E428F50CF40C38
:1001C200F513FF3EDD280430F1007408F0007108D9
:1001D2000319EF28F00D7010FF3EE9288312031374
:1001E20030307005F3007408F0007508F100F10C6E
:1001F200F00CF113F10CF00CF113700895000F30B4
:0802020097057308970408003A
:10020A00053084000008000883120313F000701000
:06021A00700880000800DE
:100220002229803083160313A2003529C030A20092
:1002300035299430A2003529D430A20035298030E8
:10024000A2003529831603132208013A0319112944
:100250002208023A031916292208033A0319192918
:100260002208043A03191C291F292303F00022083D
:10027000F0077008A2007008A6001620DD10EF013C
:100280006F0883162407840000080319512983127C
:100290006F088316240784000008A5006D20EF0A6C
:0802A00040298312DD1408005F
:1002A800053084000008000883120313F000F010E2
:0602B80070088000080040
:1002BE0083120313EF0103306F0203186F296F08C7
:1002CE00831623078400203080008312EF0A6229F0
:1002DE006F0883162307840080018312EF036F08D3
:1002EE0083162307A4000A30F4002208F000A12090
:1002FE007808F0003030F007831624088400700868
:10030E0080000A30F4002208F000A1207008831645
:10031E00A2007008003A031D952998298312EF0355
:04032E007629080024
:1003320054218316851005200520051483125D10B3
:100342000518A7295D1CA629A729A1290520052092
:10035200052005200520052005200520831685148B
:0603620005200520080043
:10036800831203137008F100F0010830FC007108D3
:10037800F40C0318C329FC0BBC29F1010034031049
:10038800C829F40C0318F107F10CF00CFC0BC52973
:0203980008005B
:0E039A00831203135F088A005E0882000800C9
:0E03A800A530FD00FD0BD62900000000080066
:1003B6008316031385140520052005140520052042
:1003C6005421831685100520052005218316051066
:0203D60008001D
:1003D8000D30FC00FB30FD00FD0BF029FC0BF02973
:1003E80000000000023083160313A2000330A300AC
:1003F8003230A40010216C08EF00EF0D6F10C920F7
:100408006C088316A2005830A3005F21583083126D
:100418000313EF00B220253083160313A5006D20C7
:020428000800CA
:10042A00013083120313ED000030EE008030831692
:10043A00A000A1012008210403194D2A0520052046
:10044A000520052005218316051005200520200812
:10045A0083126C05F000003083162105F100700844
:10046A00710403193A2A85143D2A542183168510EA
:10047A0005200520051483125D100518482A5D1C05
:10048A00472A482A422A8316A10CA00CA1131F2A24
:10049A008312ED01EE0105200520052183160510C2
:1004AA0005200520851405200520052005200514B2
:1004BA0083125D100518652A5D1C642A652A5F2A65
:1004CA00ED01EE0105200520851C6C2A6D1405201E
:1004DA0005200520052005200520052005200520EA
:1004EA0005200520052005200520052005200521D9
:1004FA008316051054218316851083126D08F000A7
:02050A000800E7
:10050C00803083120313E8000030E900EA01EB01AC
:10051C00680869040319B12A05200520831685147F
:10052C0005200520051483125D100518A12A5D1CF9
:10053C00A02AA12A9B2A851CA72A6808EA04690814
:10054C00EB04052005200521831605108312E90C08
:10055C00E80CE9138E2A83168514052005208312D6
:10056C00660867040319BD2A542183168510831667
:10057C0005200520051483125D100518C92A5D1C81
:10058C00C82AC92AC32A052005200521831605106F
:10059C000520052054218316851083126A08F0006B
:0205AC00080045
:1005AE0083120313EA016708F1000130F0007108AD
:1005BE000319E52AF00D7010FF3EDF2A7008EB00DC
:1005CE00660884000008F00570080130031D003035
:1005DE00F0006908F00603190C2B6808003C03189C
:1005EE00FC2AD421D421E803F42A660884006B087F
:1005FE000005F00070080130031D0030F00069089E
:10060E00F00603190C2BFF30EA006A08F000080010
:10061E00212B803083120313E600342BC030E6000A
:10062E00342B9430E600342BD430E600342B80305B
:10063E00E600342B831203136608013A0319102BBC
:10064E006608023A0319152B6608033A0319182B8C
:10065E006608043A03191B2B1E2B6703F00066086D
:10066E00F0077008E600DD1470088316A600162049
:0E067E00DD1068088316A6001620DD140800A3
:10068C00CD218A110A128000840ADE0A0319DF0ABE
:08069C00F003031D462B0800CA
:0C06A4008312031395011712971208002F
:1006B000CE3083120313E80001308316A2000D3000
:1006C000A3003C30A4001021EC01EC210130BB0060
:1006D00066088316A2005830A3005F2101308316FC
:1006E0000313A2000230A3005830A40010212E30C2
:1006F0008316A5006D206708003A031D882B303053
:100700008316A5006D2030308316A5006D20982B30
:1007100067088316A2005830A3005F2183120313D9
:1007200059088316A5006D205A088316A5006D2070
:100730002130EF00B220831203135708F000143069
:10074000F400B4217008EA007108EB000530F400F1
:100750005C08F000A12070086A07F4006B08031819
:10076000013EF5007508F2000030F51BFF30F30084
:100770007208E600F00170087402E700FF30E9003B
:10078000DB21C0308312EC0015226608EC00152234
:100790006708EC0015226808EC0015226908EC00D7
:0607A0001522992108005A
:1007A600831603130514851483125D100518DF2BB9
:0A07B6005D1CDE2BDF2BD92B0800A1
:1007C000831603139C1CE62B0000E02B83126608A3
:1007D00083169B008312670883169A009C131C15CE
:1007E0000B08F0008B1355309D00AA309D009C141F
:0E07F000F01BFC2B8B13FD2B8B171C1108002C
:1007FE00831603138513051306128612061386132A
:10080E0083128513051386130613861206120D2006
:10081E000D200D20861606168517052085130D2032
:10082E008517052085130D208517052085130D20AE
:10083E0006128517052085130D20851705208513B3
:10084E00861286178517052085130D20861306162A
:10085E0085170520851306128517052085130D2093
:10086E0085170520851306168517052085130D207F
:10087E000612851705208513861706178616061687
:0C088E008517052085130D20DD140800DF
:10089A00831603138611831212150C30970408006D
:1008AA0083120313660883169B009C131C141A08F0
:0408BA00F000080042
:1008BE00B626643083120313E50007309F00FF2332
:1008CE000C308316A6001620D32390308B040330F1
:1008DE00831686040516831212109210C7308316E3
:1008EE009200522301308316A2000130A30025305E
:1008FE00A40010210B30FB002630FC005D30FD0003
:10090E00FD0B872CFC0B872CFB0B872C00000000AB
:10091E0001308316A60016204D240330E600552420
:10092E0070088312E0004130FC00EE30FD00FD0B3C
:10093E009E2CFC0B9E2C00006008013A031DA82C77
:10094E00DE2C3230D700DC010130E0000930E60049
:10095E00E701E0234130FC00EE30FD00FD0BB52C2D
:10096E00FC0BB52C000001308312E6005708E7009F
:10097E00E0234130FC00EE30FD00FD0BC42CFC0BDF
:10098E00C42C000002308312E6005C08E700E0236E
:10099E004130FC00EE30FD00FD0BD32CFC0BD32CB4
:1009AE00000003308312E6006008E700E023033006
:1009BE00FB008A30FC005530FD00FD0BE42CFC0BD7
:1009CE00E42CFB0BE42C0000000001308312E60047
:1009DE00552470088312D7004130FC00EE30FD0024
:1009EE00FD0BF72CFC0BF72C00000230E600552413
:1009FE0070088312DC004130FC00EE30FD00FD0B70
:100A0E00062DFC0B062D00000930E600552470085B
:100A1E008312CB005708E6005C08E70058238312C8
:100A2E00E5036508003A031D942D6430E500DB21D3
:100A3E00C1308312EC001522E601E7018622700810
:100A4E00E10099218312611F4E2DCA0101308316D8
:100A5E00A2000D30A3004C30A40010213B08013A37
:100A6E00031D4D2DBB01E20162084B02031C4D2DEF
:100A7E006208EC00EC214130FC00EE30FD00FD0B75
:100A8E00462DFC0B462D0000E20A3B2D602DCA0AB6
:100A9E004A08053A031D602D01308316A2000D3061
:100AAE00A3005230A4001021EC01EC210130BB0058
:100ABE00CA0101305106F0007008D1007008031908
:100ACE00712D02308316A2001030A3004830A4000E
:100ADE001021792D02308316A2001030A30043306E
:100AEE00A40010214208013A031D892DC2010130D4
:100AFE00E6005708E700E02302308312E6005C08A8
:100B0E00E700E02383124108013A031D942DC10131
:100B1E000930E6004B08E700E02305308312E600BB
:100B2E000430E7000A30E800E901D7227008031903
:100B3E00B22DC50A4508033A031DA62DC501053081
:100B4E00E6000430E7000A30E800E901D722700819
:100B5E000319B22DA62D4508003A031DC72D90305E
:100B6E008B040130E6000130E7002030E8000F234F
:100B7E000230E6000130E7003E30E8000F23EF2D93
:100B8E004508013A031DDC2D90308B040230E6003F
:100B9E000130E7002030E8000F230130E60001307D
:100BAE00E7003E30E8000F23EF2D4508023A031D03
:100BBE00EF2D8B010130E6000130E7002030E80018
:100BCE000F230230E6000130E7002030E8000F234B
:100BDE004508003A031D162E4708013A031D052E3F
:100BEE00C701CB0A4B08653A031DFF2D6430CB00BD
:100BFE004B08EC00EC210130C100152E4608013ADD
:100C0E00031D152EC601CB034B08FF3A031D102EF4
:100C1E00CB014B08EC00EC210130C100582E4508E9
:100C2E00013A031D582E4708013A031D392EC701FC
:100C3E000A305C07F1007108DC007108643A031D8C
:100C4E002A2EDC01D70A5708FF3A031D302EFE303C
:100C5E00D7005708E6005C08E700582301308312DE
:100C6E00C200582E4608013A031D582EC6010A30FE
:100C7E005C02F1007108DC007108F63A031D4A2E81
:100C8E005A30DC00D70357081D3A031D502E1E3074
:100C9E00D7005708E6005C08E7005823013083129E
:060CAE00C200162D592EB4
:100CBE00FF00030E8301E3000A08E4008A017008B6
:100CCE00A0008B1C762E061C752E861C722E0130F3
:100CDE00C600C701752E0130C700C6018B10200853
:100CEE00F00064088A00630E8300FF0E7F0E090079
:100D6C0021308400363083120313F0007F30DE0014
:080D7C000630DF0046230800E9
:080CFE004D3448347A3400340F
:100D06004534633468346F3466346C34653478340F
:0A0D1600203450344C344C340034C7
:100D200050346F3477346534723420343D34203499
:020D300000348D
:020D320001348A
:0A0D3400463452344534453400348F
:020D3E0000347F
:020D400000347D
:040D42002034003425
:020D4600023475
:020D4800003475
:020D4A00003473
:040D4C002A34003411
:020D500000346D
:020D520000346B
:0A0D54004C344F3443344B34003468
:020D5E0001345E
:0A0D60004634523445344534003463
:02400E0070211F
:00000001FF
